:100000000C94D0010C9414020C9414020C9414025D
:100010000C9414020C9414020C9414020C94140208
:100020000C9414020C9414020C948F0C0C94610D1B
:100030000C9414020C9414020C9414020C941402E8
:100040000C9414020C941B210C9414020C941402B2
:100050000C9414020C94AE1A0C9414020C94140216
:100060000C9414020C9414020C9414020C941402B8
:100070000C9414020C9414020C9414020C941402A8
:100080000C9414020C9414020C9414020C94140298
:100090000C9414020C9414020C9414020C94140288
:1000A0000C9414020C9414020C941402CE0DF00D56
:1000B000DE0EF00DDE0E350E580EDE0EAD0EC00E4D
:1000C0008F118F11BE11BE11F41114124513451377
:1000D0001F124513CF12CF123613451345133F138A
:1000E000DC12DC12DC12DC12DC12DC12DC12DC12A0
:1000F000DC12DC12DC12DC12DC12DC12DC12DC1290
:10010000EE12FB1202130913131327002700270016
:1001100027002700000027002700270027002700CE
:100120002800270027002700270027002800270095
:100130002700270027002700280027002700270086
:10014000270027002800270027002700270000009D
:1001500028002700270000002700000028001E00BC
:100160001E0000001E00000028001E001E001E00D1
:100170001E00000028001E001E001E001E001E00A3
:1001800028001E001E001E001E001E0028001E006B
:100190001E001E001E001E0028001E001E001E0065
:1001A0001E001E0028001E001E001E001E001E0055
:1001B000000016034500720067006F0044006F00E6
:1001C0007800200045005A00000016034500720028
:1001D00067006F0044006F007800200045005A005F
:1001E00000000403090409026D00040100A0FA09DB
:1001F0000400000103010100092111010001223F57
:10020000000705810308000A090401000103010237
:1002100000092111010001224D0007058203080099
:100220000A09040200010300000009211101000174
:100230002236000705830308000A090403000103AE
:100240000000000921110100012239000705840383
:100250001000011201100100000008EDFE0713015B
:10026000000102000105010906A101050719E029A5
:10027000E715002501950875018102050819012976
:100280000595057501910295017503910105071901
:1002900000297715002501957875018102C00501B7
:1002A0000980A101850216010026B7001A01002A63
:1002B000B700751095018100C0050C0901A10185E9
:1002C00003160100269C021A01002A9C0275109553
:1002D000018100C005010902A1010901A100050970
:1002E0001901290515002501950575018102950162
:1002F000750381010501093009311581257F9502BA
:100300007508810609381581257F950175088106D4
:10031000050C0A38021581257F950175088106C0F4
:10032000C005010906A101050719E029E715002507
:10033000019508750181029501750881010508196B
:100340000129059505750191029501750391010536
:1003500007190029FF150025FF950675088100C0C3
:100360000000000000000000000000010204060A76
:100370000F17202C3A4A5D71879DB3C7DAE9F5FC67
:10038000FFFCF5E9DAC7B39D87715D4A3A2C201767
:100390000F0A060402010000000000000000000037
:1003A00011241FBECFEFDAE0DEBFCDBF04B603FEDF
:1003B00024C08091FB019091FC01A091FD01B091BE
:1003C000FE018730904BA740B04BB9F41092FB016F
:1003D0001092FC011092FD011092FE0114BE84B730
:1003E000877F84BF88E10FB6F894809360001092F5
:1003F00060000FBEE0E0FFE3099511E0A0E0B1E08E
:10040000E4ECF5E402C005900D92A433B107D9F7EE
:1004100011E0A4E3B1E001C01D92AB3FB107E1F7E9
:100420000E94D3090C94E0220C9400001092B900B1
:100430008AE08093B800089594EA9093BC0090916C
:10044000BC0097FFFCCF9091B900987F983021F0C5
:10045000903111F081E008958093BB0084E880938F
:10046000BC008091BC0087FFFCCF8091B900887FE1
:10047000883111F0803471F780E0089584E9809329
:10048000BC008091BC0084FDFCCF08958093BB002C
:1004900084E88093BC008091BC0087FFFCCF9091E2
:1004A000B900987F81E0983209F480E0089584E8EB
:1004B0008093BC008091BC0087FFFCCF8091BB0083
:1004C000089580910101811115C080E40E941C02F1
:1004D0008093010181110CC082E10E944602809349
:1004E0000101811105C08FEF0E9446028093010136
:1004F0000E943E0284B1807F84B985B1807F85B936
:100500008AB1837F8AB98BB1837F8BB93E98469835
:1005100008950E941C04809301010E94610280B32F
:100520008C7080BB81B3836F81BBA5E3B1E0E3E452
:10053000F1E08EE08E0F11921D928E13FCCF0C9481
:100540000604BF92CF92DF92EF92FF920F931F9318
:10055000CF93DF9380910101882379F0809134015A
:100560008F5F80933401811108C00E941C04809326
:100570000101811102C00E94AE0305E311E0C0E059
:10058000D0E0DD24D39482E0C82EEE24E394F12C55
:10059000C730D10500F580910101811164C080E46C
:1005A0000E941C0280930101811112C082E10E940D
:1005B00046028093010181110BC0C7010C2E01C0BE
:1005C000880F0A94EAF780950E9446028093010101
:1005D0000E943E0248C0CA30A1F028F4C83059F049
:1005E000C93061F005C0CC3089F070F0CD3089F0B1
:1005F000209A289810C0219A29980DC0229A2A98EA
:100600000AC0239A2B9807C0529A01C0539A5B984C
:1006100002C03E9A469890EA9A95F1F79FB179996F
:1006200002C082E001C080E091709D25982B7C99EA
:1006300002C084E001C080E0892B7D9902C038E0CF
:1006400001C030E0832B7E9902C020E101C020E090
:10065000822B9FB19095991F9927991F9295990F79
:10066000907E892B0FC080910101811149C080E4E7
:100670000E941C0280930101882379F1B12C0E9411
:100680003E028B2DF8019081981719F08083C0925B
:1006900000010E94610221960F5F1F4FCE30D105ED
:1006A00009F076CF80910001882361F18150809319
:1006B0000001882339F08FE99FE00197F1F700C02E
:1006C000000020C0A3E4B1E0E5E3F1E0CF01825FE8
:1006D00091919D938E13FCCF15C083E10E94460239
:1006E000809301018111CACF81E40E941C02809392
:1006F00001018111C3CF0E945702B82EB094BFCF21
:1007000080E0C0CF0E94AC0381E0DF91CF911F91C8
:100710000F91FF90EF90DF90CF90BF900895E82F5A
:10072000F0E0ED5BFE4F8081089508950F931F93D5
:10073000CF93DF93C3E4D1E010E00C2F025F8991E7
:1007400090E00E94241A180F0C13F9CF812FDF912B
:10075000CF911F910F9108950C946F0456985E9855
:1007600025982D9826982E9827982F988FEF90E00F
:10077000909389008093880090938B0080938A00E7
:1007800090938D0080938C00259A2D9A2FEF80E70F
:1007900092E0215080409040E1F700C00000269A8E
:1007A0002E9A2FEF80E792E0215080409040E1F7B1
:1007B00000C00000279A2F9A2FEF80E792E0215087
:1007C00080409040E1F700C0000025982D982FEF61
:1007D00080E792E0215080409040E1F700C00000A7
:1007E00026982E982FEF80E792E02150804090408D
:1007F000E1F700C0000027982F9856985E9825983A
:100800002D9826982E9827982F98089589EA8093F6
:10081000800089E08093810024982C983F988AB1C9
:100820008F748AB96E98479A8BB1806B8BB9769A20
:100830000E94AE030C946E0480E2809301018091CB
:10084000510181110EC00E94160281E08093510176
:100850002FEF83ED90E3215080409040E1F700C0FE
:10086000000080E40E941C028093010181112EC0CF
:100870000E94460280930101811128C00E94460215
:1008800080930101811122C08FE30E944602809370
:10089000010181111BC00E943E0280E40E941C02E3
:1008A00080930101811112C08CE00E944602809366
:1008B000010181110BC00E94460280930101811148
:1008C00005C08FE30E944602809301010E943E0210
:1008D00080910101089580E090E0089508950895C1
:1008E00081E0089581E008950C94720408950F93B7
:1008F0001F93CF93DF938C01FC01C081D181CE0186
:100900000E94A918BE010E942005EC01B8010E94B6
:100910007404882309F48DC0F8018281882309F4C6
:100920004AC080915D0181111FC0C431F0E5DF072D
:1009300009F051C00E94760481E080935D010E941D
:10094000781A90935C0180935B011092540110928D
:1009500056011092550110925801109257011092B1
:100960005A011092590165C080915B0190915C0120
:100970000E94841A883C910570F480915401E82FFC
:10098000F0E0EE0FFF1FEB5AFE4FD183C0838F5F65
:10099000809354014EC0C43880E5D80721F0C53893
:1009A000D04501F13AC0F8018281882341F01092CC
:1009B000520182E01EC0C438E0E5DE0759F580919F
:1009C0005201811106C086E20E94331086E20E9425
:1009D000FB1082E01CC0C438F0E5DF0741F3C538E6
:1009E000D045D9F4F8018281882331F01092530167
:1009F00080E20E944A111DC080915301811106C0FE
:100A000087E20E94331087E20E94FB1080E20E947E
:100A100051110FC0C538D04529F381E080935201B0
:100A200080935301C801DF91CF911F910F910C94D6
:100A3000700480E0DF91CF911F910F910895089588
:100A400096E0799FF001112494E5899FE00DF11D56
:100A50001124E60FF11DEE0FFF1FE65FFE4F85919B
:100A600094910895880F991FFC01E657F0408591F5
:100A700094910895880F991FFC01E65FFE4F8591C0
:100A8000949108950F931F93CF93DF93EC018115F9
:100A900020E3920750F5C11580E2D80708F0C3C0E3
:100AA000CB3BD10590F4C83AD10508F06AC0C53AED
:100AB000D10508F05BC0C430D10508F0D0C1219742
:100AC00009F0CAC101E010E00AC2CF3FD10511F020
:100AD00008F0C5C1C03FD10508F0A2C0CE01805EBC
:100AE0009109089708F4BBC1B7C1C13090E5D90797
:100AF00009F4A2C020F5C0318FE4D80770F4C11505
:100B000090E4D90708F094C0C11521E3D20708F09A
:100B1000A3C1DD278E01106CE2C1C115D04509F0DB
:100B20009BC10E94B0138FEF94E32CE08150904062
:100B30002040E1F700C000000E94D31AD0C1C115C7
:100B400097E5D90758F4C03121E5D20708F01CC158
:100B5000C43180E5D80708F475C07EC1CE01905736
:100B60008115904108F078C1DF7073C1C53AD10595
:100B700009F477C1C63AD10509F076C102E810E45C
:100B8000AEC1C83AD10509F472C1C93AD10509F418
:100B900071C1CA3AD10509F470C1CB3AD10509F443
:100BA0006FC1CC3AD10509F46EC1CD3AD10509F433
:100BB0006DC1C03BD10509F46CC1CE3AD10509F431
:100BC0006BC1CF3AD10509F46AC1C13BD10509F423
:100BD00069C1C23BD10509F468C1C33BD10509F421
:100BE00067C1C43BD10509F466C1C53BD10509F411
:100BF00065C1C63BD10509F464C1C73BD10509F401
:100C000063C1C83BD10509F462C1C93BD10509F4F0
:100C100061C1CA3BD10509F460C100E014E45FC1C1
:100C20008E0110655CC1CE019F700E943A0558C1CB
:100C3000DF708E01106A53C18091DA018160809368
:100C4000DA014DC10E94781C811102C00E945E1C15
:100C50000E94951C90E09093FB018093FA01C230B2
:100C600080E5D80721F48091FA01816086C0C43004
:100C700090E5D90721F48091FA0182607EC0C630E8
:100C800020E5D20721F48091FA01846076C0C83053
:100C900080E5D80719F48091FA0127C0CA3090E5A1
:100CA000D90721F48091FA01806167C0CC3020E53A
:100CB000D20721F48091FA0180625FC0CE3080E5D6
:100CC000D80721F48091FA01806457C0C03190E5C3
:100CD000D90721F48091FA0180684FC0C23120E524
:100CE000D20729F48091FA018460886046C0C3303D
:100CF00080E5D80721F48091FA018E7F3EC0C5308F
:100D000090E5D90721F48091FA018D7F36C0C73074
:100D100020E5D20721F48091FA018B7F2EC0C930E3
:100D200080E5D80719F48091FA0126C0CB3090E510
:100D3000D90721F48091FA018F7E1FC0CD3020E5C4
:100D4000D20721F48091FA018F7D17C0CF3080E562
:100D5000D80721F48091FA018F7B0FC0C13190E553
:100D6000D90721F48091FA018F7707C0C331D045AC
:100D700031F48091FA018B7F877F8093FA01809113
:100D8000FA010E94991CABC08D2F99278F7099276B
:100D900081309105D9F49E012370332702C0880F5A
:100DA000991F2A95E2F79C688E0144E0000F111FFD
:100DB0004A95E1F700271370802B912B53E0CC0F5D
:100DC000DD1F5A95E1F7C076DD272FC082309105EF
:100DD00031F4DC2FCC278E01016F106A80C0833084
:100DE000910569F4CE018370992701E010E002C0FB
:100DF000000F111F8A95E2F7C8019C680FC084306C
:100E00009105B9F4CE018370992701E010E002C08A
:100E1000000F111F8A95E2F7C8019A6823E0CC0FF2
:100E2000DD1F2A95E1F7C07ED7708C010C2B1D2B9E
:100E300056C08530910531F4DC2FCC278E01046F2C
:100E4000106A4DC0069709F04AC0CF71DD27DC2F2C
:100E5000CC278E01106243C000E010E040C08E013C
:100E60003EC001E810E43BC003E810E438C002EEE5
:100E700014E435C009EE14E432C00AEE14E42FC0C5
:100E800005EB14E42CC006EB14E429C007EB14E4D2
:100E900026C00CEC14E423C00DEC14E420C003E8DD
:100EA00015E41DC00AE815E41AC002E915E417C0EC
:100EB00004E915E414C001E216E411C003E216E4EB
:100EC0000EC004E216E40BC005E216E408C006E218
:100ED00016E405C007E216E402C00AE216E4C801FF
:100EE000DF91CF911F910F91089596E0799FF001C6
:100EF000112494E5899FE00DF11D1124E60FF11DE9
:100F0000EE0FFF1FE65FFE4F85919491803E9105A5
:100F1000E0F4803C910558F58133910509F46FC0E8
:100F200048F48932910509F463C08A32910509F4C5
:100F30006DC072C089339105E9F082389105D1F016
:100F40008533910509F44DC067C0833E910581F159
:100F500038F4803E9105B9F0823E9105D9F05CC02D
:100F6000863E910561F1873E9105A1F155C00E9431
:100F7000320508952091FA0120FD02C021FF4CC0E6
:100F800080EE90E049C08091FA0180FFF9CF89E3BB
:100F900090E042C08091FA0182FF0EC08091FA0178
:100FA00084FF03C080E090E037C083EE90E034C05F
:100FB0008091FA0182FFF2CF82EE90E02DC0809105
:100FC000FA0183FF0BC08091FA0184FDEBCF87EE1D
:100FD00090E022C08091FA0183FFF5CF86EE90E089
:100FE0001BC08091FA0185FF07C089E290E014C020
:100FF0008091FA0185FFF9CF85E390E00DC08091E3
:10100000FA0186FF07C08AE290E006C08091FA01EB
:1010100086FFF9CF81E390E00E944205089508958C
:101020000C940F0880916E010895CF93DF9300D048
:101030001F92CDB7DEB79C018091F101843019F584
:1010400093E099833B832A839093E9008FEF9091FB
:10105000E800815095FD06C095ED9A95F1F70000E6
:101060008111F5CF8091E80085FF0DC040E050E090
:1010700063E070E0CE0101960E947F0A8091E80053
:101080008E778093E8000F900F900F90DF91CF91B3
:101090000895CF93DF9300D01F92CDB7DEB7209194
:1010A000F101243021F522E029839B838A8383E0A8
:1010B0008093E9008FEF9091E800815095FD06C084
:1010C00095ED9A95F1F700008111F5CF8091E80038
:1010D00085FF0DC040E050E063E070E0CE01019676
:1010E0000E947F0A8091E8008E778093E8000F903D
:1010F0000F900F90DF91CF9108952091F10124304E
:10110000F1F422E02093E9002FEF3091E800215024
:1011100035FD06C035ED3A95F1F700002111F5CF08
:101120002091E80025FF0BC040E050E065E070E052
:101130000E947F0A8091E8008E778093E8000895EE
:10114000CF93DF93EC019091F101943009F046C008
:1011500080910C018823D9F080910D018823B9F08A
:101160009093E9008FEF9091E800815095FD06C0C3
:1011700095E19A95F1F700008111F5CF8091E80093
:1011800085FF2CC040E050E060E170E017C081E0D6
:101190008093E9008FEF9091E800815095FD06C0A3
:1011A00095ED9A95F1F700008111F5CF8091E80057
:1011B00085FF14C040E050E068E070E0CE010E947E
:1011C0007F0A8091E8008E778093E80080E1FE013D
:1011D000AEE5B1E001900D928A95E1F7DF91CF91F4
:1011E00008958091F001811109C00E94140C0E94A1
:1011F000710C8091E20084608093E2000895109267
:10120000F001089508950C9408210E94691A0E9423
:101210000E210E94170F0C94100842E061EC81E04F
:101220000E948E0B42E061EC82E00E948E0B42E055
:1012300061EC83E00E948E0B42E161EC84E00C944F
:101240008E0B8091F301833009F455C030F4813066
:1012500071F0823009F48EC008958A3009F47AC0A2
:101260008B3009F460C0893009F09CC020C08091A7
:10127000F201813A09F096C08091E800877F80935F
:10128000E8008091F6019091F701892B21F460E14B
:101290008EE591E003C060E080E090E070E00E94A5
:1012A000CA0A8091E8008B778093E80008958091C6
:1012B000F201813209F076C08091F6019091F70138
:1012C000009719F0039709F06DC08091E800877FBF
:1012D0008093E8008091E80082FD05C08091F101D3
:1012E0008111F8CF5FC08091F10080936E018091F1
:1012F000E8008B7753C08091F201813A09F052C027
:101300008091F6019091F701892B09F04BC08091F3
:10131000E800877F8093E8008091E80080FFFCCFA1
:1013200080910C0136C08091F2018132D9F5809113
:10133000F6019091F701892BA9F58091E800877F4C
:101340008093E8000E94C30B8091F40180930C010C
:101350000C94B0138091F201813221F58091E80064
:10136000877F8093E8000E94C30B8091F5018093F2
:101370006F0108958091F201813AA1F48091E80013
:10138000877F8093E8008091E80080FFFCCF809108
:101390006F018093F1008091E8008E778093E800E0
:1013A0000C94C30B089584B7877F84BF88E10FB680
:1013B000F89480936000109260000FBE90E080E887
:1013C0000FB6F89480936100909361000FBE0E9465
:1013D000660F0E94140C0E94710C8091E2008460E0
:1013E0008093E20078940E94F70E0E94680F82E0DA
:1013F00091E00E94120F0E94F6208091F101853049
:1014000069F40E94301A8091EF018823B1F30E94A1
:101410005B1A882391F30E94690AEFCF0E946E0F36
:10142000ECCF292F332723303105C9F064F4213064
:10143000310581F02230310509F043C08DE690E09E
:1014400026EE31E042C021323105F1F02232310581
:1014500041F137C082E190E023E532E036C09927C0
:101460008130910541F08230910541F0892B49F599
:10147000E2EEF1E005C0EAECF1E002C0E2EBF1E0FF
:10148000849190E09F0121C06430D8F4E62FF0E011
:10149000EE0FFF1FEE5DFE4F2081318189E090E06D
:1014A00014C0643070F470E0FB01EE0FFF1FE65EC5
:1014B000FE4F20813181FB01EA5EFE4F808190E08A
:1014C00004C080E090E020E030E0FA013183208326
:1014D000089580E189BD82E189BD09B400FEFDCF98
:1014E0008091D8008F7D8093D8008091E000826049
:1014F0008093E0008091E00081FDFCCF0895CF92C1
:10150000DF92EF92FF920F931F93CF93DF93EC0143
:101510008B016A010E94E20B811133C0C114D10416
:1015200039F0F60180819181081B190BC80FD91F72
:10153000E12CF12C0115110519F18091E80085FDD0
:1015400016C08091E8008E778093E800C114D10422
:1015500049F0F60180819181E80EF91EF182E08266
:1015600085E00FC00E94E20B882321F30AC0899115
:101570008093F10001501109FFEFEF1AFF0ADACF53
:1015800080E0DF91CF911F910F91FF90EF90DF905E
:10159000CF9008952091F8013091F901261737076F
:1015A00048F06115710539F42091E8002E772093F9
:1015B000E80001C0B90140E061157105A9F1209171
:1015C000F101222309F443C0253009F442C02091DF
:1015D000E80023FD40C02091E80022FD32C02091A8
:1015E000E80020FFE9CF4091F3002091F20030E0C5
:1015F000342BFC01CF016115710559F028303105FC
:1016000040F481918093F100615071092F5F3F4F49
:10161000F1CF41E02830310509F040E02091E800A9
:101620002E772093E800C8CF4111C9CF0AC080911E
:10163000F101882361F0853061F08091E80083FD3D
:101640000AC08091E80082FFF2CF80E0089582E036
:10165000089583E0089581E008952091F801309184
:10166000F9012617370748F06115710539F4209103
:10167000E8002E772093E80001C0B901FC0120E0CA
:101680006115710591F18091F101882309F440C041
:10169000853009F43FC08091E80083FD3DC0809112
:1016A000E80082FD2FC08091E80080FFE9CF209103
:1016B000F3008091F20090E0922B6115710559F0D2
:1016C0008830910540F424912093F10031966150C7
:1016D00071090196F2CF21E0089709F020E080918E
:1016E000E8008E778093E800CBCF2111CCCF0AC0E1
:1016F0008091F101882361F0853061F08091E800EC
:1017000083FD0AC08091E80082FFF2CF80E0089557
:1017100082E0089583E0089581E00895982F97303E
:1017200058F59093E900981739F07091EC002091EA
:10173000ED005091F00003C0242F762F50E021FFE0
:1017400019C03091EB003E7F3093EB003091ED00FB
:101750003D7F3093ED003091EB0031603093EB0032
:101760007093EC002093ED005093F0002091EE0078
:1017700027FF07C09F5FD3CF8F708093E90081E080
:10178000089580E008958091F20187FF11C0809153
:10179000E80082FD05C08091F1018111F8CF11C0F0
:1017A0008091E8008B770BC08091F101882349F08C
:1017B0008091E80080FFF8CF8091E8008E778093D9
:1017C000E80008952091E4003091E50095E640910D
:1017D000EC00842F817040FF22C08091E80080FDE2
:1017E0001CC08091F101882391F0853091F08091A7
:1017F000EB0085FD10C04091E4005091E5004217D8
:10180000530729F39A01915011F784E0089582E07B
:10181000089583E0089581E0089580E0089540915F
:10182000E80042FFDECF08950E94820C0E948A0CDD
:10183000E0EEF0E0808181608083E8EDF0E080817F
:101840008F77808319BCA7EDB0E08C918E7F8C934D
:1018500080818F7E80831092F00108950F931F93F3
:10186000CF93DF930E94820C0E948A0CC8EDD0E0D7
:1018700088818F77888388818068888388818F7D3D
:10188000888319BC1092F1011092ED011092EF01C2
:101890001092EE0100EE10E0F80180818B7F8083D2
:1018A00088818160888342E060E080E00E948E0B46
:1018B000E1EEF0E080818E7F8083E2EEF0E08081D7
:1018C00081608083808188608083F80180818E7F41
:1018D0008083888180618883DF91CF911F910F91F0
:1018E0000895E8EDF0E080818F7E8083E7EDF0E001
:1018F00080818160808384E082BF81E08093F001F9
:101900000C942E0CE8EDF0E080818E7F80831092A5
:10191000E20008951092DA001092E10008951F92FB
:101920000F920FB60F9211242F933F934F935F9313
:101930006F937F938F939F93AF93BF93EF93FF9397
:101940008091E10082FF0BC08091E20082FF07C01E
:101950008091E1008B7F8093E1000E94F60E8091E0
:10196000DA0080FF1FC08091D80080FF1BC08091EB
:10197000DA008E7F8093DA008091D90080FF0DC05D
:1019800080E189BD82E189BD09B400FEFDCF81E01F
:101990008093F1010E94F10805C019BC1092F10179
:1019A0000E94FF088091E10080FF19C08091E20051
:1019B00080FF15C08091E2008E7F8093E2008091CD
:1019C000E20080618093E2008091D8008062809381
:1019D000D80019BC85E08093F1010E940309809131
:1019E000E10084FF30C08091E20084FF2CC080E1E0
:1019F00089BD82E189BD09B400FEFDCF8091D80088
:101A00008F7D8093D8008091E1008F7E8093E100EC
:101A10008091E2008F7E8093E2008091E2008160FD
:101A20008093E2008091ED01882311F084E007C0EB
:101A30008091E30087FD02C081E001C083E08093D4
:101A4000F1010E9405098091E10083FF29C0809186
:101A5000E20083FF25C08091E100877F8093E10051
:101A600082E08093F1011092ED018091E1008E7F80
:101A70008093E1008091E2008E7F8093E20080916C
:101A8000E20080618093E20042E060E080E00E943A
:101A90008E0B8091F00088608093F0000E94020914
:101AA000FF91EF91BF91AF919F918F917F916F9136
:101AB0005F914F913F912F910F900FBE0F901F900C
:101AC00018951F920F920FB60F9211242F933F93E8
:101AD0004F935F936F937F938F939F93AF93BF9336
:101AE000CF93DF93EF93FF93C091E900CF70809184
:101AF000EC00D82FD17080FDD0E81092E9008091E1
:101B0000F000877F8093F00078940E94A50D1092DA
:101B1000E9008091F00088608093F000CD2BCF70B9
:101B2000C093E900FF91EF91DF91CF91BF91AF9109
:101B30009F918F917F916F915F914F913F912F91E5
:101B40000F900FBE0F901F9018951F93CF93DF93A8
:101B5000CDB7DEB7AA970FB6F894DEBF0FBECDBFE4
:101B6000E2EFF1E088E08E0F9091F10091938E13F7
:101B7000FBCF0E9421098091E80083FF1FC1809163
:101B8000F2019091F301492F50E04A30510508F0DD
:101B900015C1FA01EA5AFF4F0C949022803881F067
:101BA000823809F00BC18091F6018F708093E900B3
:101BB0008091EB0085FB882780F91092E90006C030
:101BC0008091EE019091EF01911182609091E80077
:101BD000977F9093E8008093F1001092F100C8C0C5
:101BE000282F2D7F09F0EAC0882319F0823061F098
:101BF000E5C08091F401813009F0E0C0933009F034
:101C000080E08093EF012BC08091F401811127C007
:101C10008091F6018F7009F4D1C08093E900209182
:101C2000EB0020FF1CC0933021F48091EB00806218
:101C300014C09091EB0090619093EB0021E030E0B4
:101C4000A90102C0440F551F8A95E2F74093EA00AC
:101C50001092EA008091EB0088608093EB00109274
:101C6000E9008091E800877F86C08111A7C01091AC
:101C7000F4011F778091E3008078812B8093E3004B
:101C80008091E800877F8093E8000E94C30B8091D9
:101C9000E80080FFFCCF8091E30080688093E30040
:101CA000111102C082E001C083E08093F10186C07F
:101CB0008058823008F082C08091F4019091F50143
:101CC0008C3D53E0950779F583E08A838AE2898326
:101CD0004FB7F894DE01139620E03EE051E2E32F87
:101CE000F0E050935700E49120FF03C0E295EF70BD
:101CF0003F5FEF708E2F90E0EA3010F0C79601C082
:101D0000C0968D939D932F5F243149F74FBF8091EB
:101D1000E800877F8093E8006AE270E0CE010196D8
:101D20000E94CA0A14C0AE014F5F5F4F6091F60176
:101D30000E94110ABC01009709F440C09091E8008C
:101D4000977F9093E80089819A810E942D0B809162
:101D5000E8008B778093E80031C0803879F5809176
:101D6000E800877F8093E8008091ED018093F10087
:101D70008091E8008E778093E8000E94C30B1EC01C
:101D800081111CC09091F4019230C0F48091E80060
:101D9000877F8093E8009093ED010E94C30B8091B0
:101DA000ED01811106C08091E30087FD02C081E052
:101DB00001C084E08093F1010E940D098091E80048
:101DC00083FF0AC08091E800877F8093E8008091BC
:101DD000EB0080628093EB00AA960FB6F894DEBF0A
:101DE0000FBECDBFDF91CF911F9108950895CF937E
:101DF0008091F1018823A1F0C091E900CF7090910A
:101E0000EC00892F817090FD80E8C82B1092E900CA
:101E10008091E80083FD0E94A50DCF70C093E9007A
:101E2000CF91089590937501809374010895E09186
:101E30007401F0917501309721F00190F081E02D4F
:101E4000099480E00895E0917401F0917501309754
:101E500021F00280F381E02D09940895E09174014E
:101E6000F0917501309721F00480F581E02D0994FF
:101E7000089520917201309173018217930771F0D8
:101E80009093730180937201E0917401F091750158
:101E9000309721F00680F781E02D09940895209174
:101EA0007001309171018217930771F09093710165
:101EB00080937001E0917401F0917501309721F0E9
:101EC0000084F185E02D0994089508950C94650F20
:101ED0000E946F1A0E9489020C94311B9F92AF924C
:101EE000BF92CF92DF92EF92FF920F931F93CF9307
:101EF000DF9300D000D000D0CDB7DEB70E94A102A2
:101F00000DE010E0AA24A394B12C902E802F0E9403
:101F10008F03980129583E4F6901F901F080F82696
:101F2000A1F40150110988F78FEF89838A831B82FE
:101F30000E94781A8160782F9D838C8349815A8111
:101F40006B818D810E9405102FC09091DA0191FF65
:101F500004C08E830E9495038E8125E030E0A501A8
:101F6000022E01C0440F0A94EAF7E42E4F21C1F07B
:101F700029839A828E2191E009F490E09B830E944C
:101F8000781A8160782F9D838C8349815A816B8177
:101F90008D810E940510F6018081E826E08204C050
:101FA00021503109E0F6BDCF0E94181E1091760134
:101FB0000E94170F1817B9F00E94170F809376012F
:101FC00026960FB6F894DEBF0FBECDBFDF91CF913E
:101FD0001F910F91FF90EF90DF90CF90BF90AF9047
:101FE0009F900C94100826960FB6F894DEBF0FBE93
:101FF000CDBFDF91CF911F910F91FF90EF90DF90B8
:10200000CF90BF90AF909F900895CF93DF93CDB7BF
:10201000DEB72B970FB6F894DEBF0FBECDBF4F8350
:10202000588769877A878B87DE01119686E0FD01E4
:1020300011928A95E9F785E0FE01379601900D929D
:102040008A95E1F749815A816B817C818D819E81DE
:102050000E944E162B960FB6F894DEBF0FBECDBF72
:10206000DF91CF910895CF93882309F4C2C0C82F80
:10207000823859F40E94170F81FDBBC089E30E948A
:1020800028190E94F51989E30CC0833879F40E945D
:10209000170F80FDAEC083E50E9428190E94F51934
:1020A00083E50E946A19CF910C94F519843859F48C
:1020B0000E94170F82FD9DC087E40E9428190E948C
:1020C000F51987E4EECF8CEF8C0F813A48F48C2F12
:1020D0000E945B2081118DC08C2F0E942819E3CFB4
:1020E00080E28C0F883048F4C77081E001C0880F0F
:1020F000CA95EAF70E94AE19D6CF8BE58C0F8330D4
:1021000078F4C53A29F0C63A31F083E890E005C08A
:1021100081E890E002C082E890E0CF910C94390F02
:1021200088E58C0F833108F064C0C83A39F1C93AA8
:1021300041F1CA3A49F1CB3A51F1CC3A59F1CD3A91
:1021400061F1C03B69F1CE3A71F1CF3A79F1C13B0F
:1021500081F1C23B89F1C33B91F1C43B99F1C53B8D
:10216000A1F1C63BA9F1C73BB1F1C83BB9F1C93BED
:10217000C1F1CA3BC9F180E090E038C082EE90E046
:1021800035C089EE90E032C08AEE90E02FC085EB3A
:1021900090E02CC086EB90E029C087EB90E026C051
:1021A0008CEC90E023C08DEC90E020C083E891E0BF
:1021B0001DC08AE891E01AC082E991E017C084E965
:1021C00091E014C081E292E011C083E292E00EC07F
:1021D00084E292E00BC085E292E008C086E292E0E1
:1021E00005C087E292E002C08AE292E0CF910C94AF
:1021F0004F0FCF910895882309F44BC0823859F4CA
:102200000E94170F81FF45C089E30E9428190E9490
:10221000F51989E30CC0833871F40E94170F80FF11
:1022200038C083E50E9428190E94F51983E50E94B1
:102230006A190C94F519843859F40E94170F82FF1B
:1022400028C087E40E9428190E94F51987E4EFCF7F
:102250009CEF980F913A58F390E2980F983050F411
:10226000877091E001C0990F8A95EAF7892F0E9443
:10227000B419DFCF9BE5980F933020F480E090E015
:102280000C94390F885A833120F480E090E00C944C
:102290004F0F0895882321F00E94AE190C94F51970
:1022A0000895882321F00E94B4190C94F51908951B
:1022B0007F928F929F92AF92BF92CF92DF92EF92D6
:1022C000FF920F931F93CF93DF931F92CDB7DEB78B
:1022D0007C01C62E772EFC01058102950F701281BC
:1022E00011110E94CB190E942119882379F0112322
:1022F00069F080E28C0D883048F082E00E940A1973
:102300000E94211991E0D82ED92601C0D12CE72DA9
:10231000E295EF70F0E0E05AFF4F0C949022872D89
:10232000807F072D0F70882311F00295007F112305
:1023300089F0002309F490C180E28C0D883020F4EC
:10234000802F0E94AE1903C0802F0E94BE190E94E8
:10235000F51982C18C2D0E94FB10002309F495C150
:1023600080E28C0D883020F4802F0E94B41903C0C5
:10237000802F0E94C4190E94F51987C1972D907F64
:10238000872D8F70903211F08295807FCC2021F0C4
:10239000F1E0CF16B1F01EC0112349F0002309F47B
:1023A00014C1013009F011C10E94DE196EC1002371
:1023B00019F0013009F469C189830E94E11989810A
:1023C0000AC1112321F0023008F05FC1FEC00111E3
:1023D0005CC101C1112321F0002309F4F6C03CC106
:1023E000002309F4F8C03EC1872D86958695837039
:1023F00090E0009719F0019761F047C1112321F097
:102400008C2D972D937002C080E090E00E94390FD0
:102410003CC1112321F08C2D972D937002C080E0D8
:1024200090E00E944F0F31C18C2D112319F00E94B2
:10243000201D02C00E94881D0E940D1E26C1872DEE
:10244000837009F052C0111120C18C2D82958695A0
:102450008770880F880F9C2D9F70892E912CA12C3E
:10246000B12C082E04C0880C991CAA1CBB1C0A9411
:10247000D2F7C4FE14C00FE010E020E030E0B90154
:10248000A80104C0440F551F661F771F8A95D2F715
:10249000CB01BA01609570958095909503C060E07E
:1024A00070E0CB01272D26952695237030E0223051
:1024B000310569F02330310589F0682979298A29A5
:1024C0009B292130310571F00E949617DEC06829E2
:1024D00079298A299B290E94B217D7C00E94961792
:1024E000C501B4010E947A17D0C0112319F0872DBD
:1024F000817001C08695882309F4C7C08C2D829510
:1025000086958770880F880F9C2D9F70892E912C3F
:10251000A12CB12C082E04C0880C991CAA1CBB1C31
:102520000A94D2F7C4FE14C00FE010E020E030E0BF
:10253000B901A80104C0440F551F661F771F8A9573
:10254000D2F7CB01BA01609570958095909503C044
:1025500060E070E0CB01272D269526952370422F51
:1025600050E04230510569F04330510589F0682947
:1025700079298A299B294130510571F00E947018F0
:1025800084C0682979298A299B290E948C187DC0DA
:102590000E947018C501B4010E94541876C08C2D99
:1025A00090E0FC01E05EF109E531F10508F050C072
:1025B000E059FF4F0C9490220C2D0F70872D8F71D6
:1025C000112331F00E94ED17802F0E944A115DC047
:1025D0000E940E18802F0E94511157C0112339F00C
:1025E000011153C0872D8F710E9433184EC00230E5
:1025F00008F04BC0F7CF112339F0872D8F710E945F
:10260000ED1743C01123C9F3872D8F710E940E1857
:102610003CC0112329F0872D8F710E94D81735C037
:102620000E94CE1732C0112351F0172D1F71812F38
:102630000E94ED1763E0812F0E94011926C081E0FE
:102640000E940A19023008F182E00E940A191DC096
:10265000112331F0002389F28C2D0E94331015C014
:10266000002391F28C2D0E94FB100FC0472D4F705C
:102670006C2DC7010E946B040E94F21606C0472D04
:102680004F706C2DC7010E941F05DD20F9F00E94DC
:10269000FD1880FD1BC0F70112820E94F7180E94EE
:1026A000ED17C7010E9475130E94F7180F90DF9174
:1026B000CF911F910F91FF90EF90DF90CF90BF903F
:1026C000AF909F908F907F900C940E180F90DF9199
:1026D000CF911F910F91FF90EF90DF90CF90BF901F
:1026E000AF909F908F907F9008950F931F93CF93FB
:1026F000DF93EC01888199812B813C81232BB9F0F8
:102700009F3F11F48F3F99F0CE010E9477048823F8
:1027100071F0688179818A810E94F3188C010E948E
:10272000A8180E946F17B801CE010E945811DF91BE
:10273000CF911F910F9108950E94CB190E94DB1930
:102740000E94A0190E94F5190E94BE1E0E940D1E33
:1027500080E090E00E94390F80E090E00C944F0FF1
:102760000E94BB190C949C130E94E818292F2295F3
:102770002F7030E02C3031054CF42A3031056CF4E8
:102780002250310922303105A8F407C02C30310520
:1027900069F02F30310551F00DC0803F69F018F419
:1027A000803E40F409C0843F29F406C093FB88278B
:1027B00080F9089580E0089581E00895CF93DF9334
:1027C00000D000D01F92CDB7DEB70F900F900F90C2
:1027D0000F900F90DF91CF910895CF93DF9300D0AA
:1027E00000D000D0CDB7DEB726960FB6F894DEBF86
:1027F0000FBECDBFDF91CF9108951F93CF93DF938D
:10280000C091850116E080918601C81799F0D0E04B
:102810001C9FF0011D9FF00D1124E957FE4F4081D0
:10282000518162817381848195810E94ED1321968B
:10283000C770E9CFDF91CF911F9108954091B70103
:102840005091B8016091B9017091BA018091BB01BA
:102850009091BC010C94ED138091BC0182958F7016
:1028600009F054C08091B901882309F44FC08091C8
:102870008501A09186016091B7017091B8014091E6
:10288000BA015091BB01B6E08A1709F43FC090E04D
:1028900041155105C1F17F3F11F46F3FA1F1B89F80
:1028A000F001B99FF00D1124E957FE4F21817213F9
:1028B0002AC02081621327C02281211124C02381D4
:1028C00034812417350710F421503109241B350BAE
:1028D000283C3105C0F42091BC012F702061209369
:1028E000BC0126E0289FF001299FF00D1124E45738
:1028F000FE4F80818F708061808387EB91E00E9422
:1029000075130C94FD1301968770BECF0895CF9276
:10291000DF92EF92FF920F931F93CF93DF93CDB788
:10292000DEB762970FB6F894DEBF0FBECDBF8C0145
:1029300085E0F801DE011D9601900D928A95E1F780
:10294000D8014C9111965C91119712966C91129747
:102950001396CD90DC9014973091B7017091B80127
:102960008091BA019091BB01009709F46BC17F3F40
:1029700019F43F3F09F466C1E090B901EE2009F473
:10298000C0C02091BC01C816D90628F0F601E81B8A
:10299000F90BCF0104C0809590958C0D9D1DFF24EF
:1029A000F394883C910578F0F12C207F09F0C6C0A3
:1029B0007C2DD98AC88A89890E94DE1387EB91E031
:1029C0000E947513B1C0822F807F09F046C0751335
:1029D00014C0341312C0611110C02F7020612093F5
:1029E000BC010E941E1487EB91E00E947513809138
:1029F000BC01D80115968C932EC0CD2819F15F3FEC
:102A000011F44F3FF9F0F62E61111CC08091850141
:102A10002091860136E0821709F45AC090E0389F71
:102A2000F001399FF00D1124E957FE4F71815713C2
:102A300006C07081471303C07281711103C00196F3
:102A40008770E9CFF62E662309F418C18091BC0186
:102A500081608093BC01F12C11C1751308C034133F
:102A600006C0611104C08091BC01D801C3C04D876C
:102A70005E878D859E856A8B0E94B4136A89882340
:102A8000E1F16623D1F12091BC01822F82958F70F4
:102A900090E0029774F08091B7019091B801988707
:102AA0008F831986DB86CA862C87CE0107960E9403
:102AB000751386E0F801A7EBB1E001900D928A95BD
:102AC000E1F70E942C140E941E14FF24F394D6C038
:102AD0004D875E878D859E850E94E818292F229557
:102AE0002F7030E0223031050CF0BCC09F7009F02F
:102AF000B6C0805E883008F4C1C0C8010E9475135A
:102B0000E4CFC816D90608F453C0F601E81BF90B48
:102B1000CF01883C910508F450C0F12C7C2DD98A56
:102B2000C88A89890E94DE13E7EBF1E086E0DF01C5
:102B30001D928A95E9F70E941E14A0C0751314C057
:102B4000341312C0611110C08091BC01F80185835B
:102B5000C8010E94751386E0E7EBF1E0DF011D92EA
:102B60008A95E9F7FE2C8AC04D875E878D859E8504
:102B70006A8B0E94B4136A89882309F4BECF662346
:102B800009F4BBCF2091BC01822F82958F7090E019
:102B900002970CF48ECF8091B7019091B8019A837F
:102BA00089831B82DD82CC822E83CE0101967FCF6A
:102BB000809590958C0D9D1DACCFF62E662309F463
:102BC0009CCF75132EC034132CC02091BC0120FD66
:102BD0001FC0822F82958F70D9F0D80115962C9343
:102BE00015978F3049F08F5F982F9295907F822FA5
:102BF0008F70892B15968C93C8010E94751386E0FF
:102C0000F801A7EBB1E001900D928A95E1F793CF1F
:102C100086E0F801A7EBB1E001900D928A95E1F70B
:102C20002DC04D875E878D859E850E94B4138111CE
:102C300040CF8091BC0181608093BC01C8010E949B
:102C400075131CC0662309F458CF4D875E878D85A8
:102C50009E850E94B413882309F44FCF2ACF811197
:102C600048CF0CC0243031050CF047CF9F7009F4D9
:102C700040CFF8019581907F09F03BCF8F2D629670
:102C80000FB6F894DEBF0FBECDBFDF91CF911F917D
:102C90000F91FF90EF90DF90CF9008951F93CF9307
:102CA000DF93CDB7DEB72C970FB6F894DEBF0FBE1B
:102CB000CDBF4F83588769877A878B879C87CE01E2
:102CC00007960E948714882369F08F8198852A854A
:102CD0003B85232BF1F19F3F09F063C08F3F09F043
:102CE00060C037C086E0FE013796DE011196019084
:102CF0000D928A95E1F76F817885EA85FB8530979B
:102D000041F17F3F11F46F3F21F12091860130E0C6
:102D1000C9010196877099274091850150E0841779
:102D2000950709F447C069837A83FD83EC8396E0B5
:102D3000929FD001939FB00D1124A957BE4FFE0161
:102D4000319601900D929A95E1F7809386010E9449
:102D5000FD1316E080918501909186018917C1F1DC
:102D6000189FC001112489579E4F0E948714882301
:102D700079F1E09185011E9FF0011124E957FE4F82
:102D80004081518162817381848195810E94ED131C
:102D90008091850190E00196877099278093850145
:102DA000D9CF4F81588569857A858B859C850E940E
:102DB000ED13CFCF0E94B0131092860110928501BF
:102DC000E7EBF1E086E0DF011D928A95E9F7C1CFDC
:102DD0002C960FB6F894DEBF0FBECDBFDF91CF911A
:102DE0001F910895EF92FF920F931F93CF93DF935C
:102DF0008C01009709F46CC0F12CEE24E394E801F7
:102E00002196F8018491843740F4843008F051C051
:102E1000813081F0823019F15BC0853709F444C0FC
:102E2000A8F19CE7980F903708F052C08F770E9466
:102E3000FB1041C00E5F1F4FFE01C49180E28C0F5A
:102E4000883048F4C7708E2D01C0880FCA95EAF704
:102E50000E94CE1914C08C2F0E9433102DC00E5F1B
:102E60001F4FFE01C49180E28C0F883058F4C77068
:102E70008E2D01C0880FCA95EAF70E94D4190E94CE
:102E8000F5191AC08C2F0E94FB1016C00E5F1F4F41
:102E9000FE01C491CC2381F08FE99FE00197F1F707
:102EA00000C00000C150F6CF0E5F1F4FFE01F4902E
:102EB00003C00E9433108E018F2D882309F49FCF09
:102EC000EFE9FFE03197F1F700C000008150F5CF46
:102ED000DF91CF911F910F91FF90EF90089508958A
:102EE0006093C1017093C2018093C3019093C401A8
:102EF0000C949C130F931F930091C1011091C20178
:102F00002091C3013091C401DC01CB01802B912BB6
:102F1000A22BB32B8093C1019093C201A093C30154
:102F2000B093C4011F910F910C949C130F931F93A6
:102F30000091C1011091C2012091C3013091C401DF
:102F4000DC01CB0180239123A223B3238093C10111
:102F50009093C201A093C301B093C4011F910F913C
:102F60000C949C130F931F930091C1011091C20107
:102F70002091C3013091C401DC01CB01802791274E
:102F8000A227B3278093C1019093C201A093C301EC
:102F9000B093C4011F910F910C949C131092BD012A
:102FA0001092BE011092BF011092C0010C949C13AC
:102FB00041E050E060E070E004C0440F551F661F20
:102FC000771F8A95D2F74093BD015093BE0160935D
:102FD000BF017093C0010C949C1341E050E060E08D
:102FE00070E004C0440F551F661F771F8A95D2F703
:102FF0008091BD019091BE01A091BF01B091C0012F
:10300000482B592B6A2B7B2B4093BD015093BE015B
:103010006093BF017093C0010C949C1341E050E099
:1030200060E070E004C0440F551F661F771F8A954B
:10303000D2F740955095609570958091BD01909123
:10304000BE01A091BF01B091C001482359236A235A
:103050007B234093BD015093BE016093BF017093E9
:10306000C0010C949C1341E050E060E070E004C0AB
:10307000440F551F661F771F8A95D2F78091BD01B7
:103080009091BE01A091BF01B091C001482759277E
:103090006A277B274093BD015093BE016093BF0117
:1030A0007093C0010C949C130F931F930091BD016A
:1030B0001091BE012091BF013091C001DC01CB0114
:1030C000802B912BA22BB32B8093BD019093BE013B
:1030D000A093BF01B093C0011F910F910C949C135A
:1030E0000F931F930091BD011091BE012091BF016C
:1030F0003091C001DC01CB0180239123A223B323B3
:103100008093BD019093BE01A093BF01B093C00115
:103110001F910F910C949C130F931F930091BD016D
:103120001091BE012091BF013091C001DC01CB01A3
:1031300080279127A227B3278093BD019093BE01DA
:10314000A093BF01B093C0011F910F910C949C13E9
:103150000895CF92DF92EF92FF920F931F93CF9338
:10316000DF938C01C090C101D090C201E090C301F7
:10317000F090C4018091BD019091BE01A091BF016A
:10318000B091C001C82AD92AEA2AFB2ACFE1D0E0AF
:10319000D701C6010C2E04C0B695A79597958795C3
:1031A0000A94D2F780FF06C0B8018C2F0E947507E1
:1031B000019721F4219760F780E001C08C2FDF9107
:1031C000CF911F910F91FF90EF90DF90CF900895D6
:1031D000CF93DF93EC010E94A918BE010E947507EE
:1031E000DF91CF910895CB010E94E8180895809156
:1031F000C50185958595859508958091C501877050
:10320000089598E0899F90011124262B2093C501F1
:103210000C94ED172091C501809582238093C50100
:10322000982F977069F430E0482F552747FD509547
:103230002417350729F08595859585950C940E18EA
:1032400008959091C501977081E009F480E0089598
:1032500090910C01992321F090910D01911109C0D9
:1032600020910E0130910F01F90132969FEF40E05D
:103270001FC0982F9695969596959F3050F5E091A2
:103280000E01F0910F01E90FF11D877021E030E090
:10329000A90102C0440F551F8A95E2F7CA01918126
:1032A000892B818308959F3F39F04F5F4E3041F065
:1032B00051915813F8CF0DC05111F7CF942FF5CF7E
:1032C0009F3F39F0F901E90FF11D97FDFA958283CF
:1032D0000895089590910C01992321F090910D018A
:1032E000911109C020910E0130910F01F901329620
:1032F000205F3F4F1FC0982F9695969596959F30CB
:10330000F0F4E0910E01F0910F01E90FF11D8770CB
:1033100021E030E0A90102C0440F551F8A95E2F771
:10332000CA01809591818923818308953196E2179E
:10333000F30729F090819813F9CF1082F7CF089501
:1033400081E090E0E0910E01F0910F01E80FF91F8C
:103350001082019680319105A9F708959091D901C5
:10336000892B8093D901089580959091D901892363
:103370008093D90108951092D90108959091D801B0
:10338000892B8093D801089580959091D801892345
:103390008093D80108951092D80108959091D70193
:1033A000892B8093D701089580959091D701892327
:1033B0008093D70108951092D70108958093C60194
:1033C00008951092C601089580910E0190910F0109
:1033D000FC0131969C01205F3F4F80E0919191115B
:1033E0008F5FE217F307D1F70895E0910E01F09196
:1033F0000F018091D9018083E0910E01F0910F01BE
:1034000090818091D801892B8083E0910E01F09109
:103410000F0190818091D701892B80838091C60113
:10342000882361F0E0910E01F0910F019081892BCA
:1034300080830E94E41981111092C60180910E01CF
:1034400090910F010C94230F20E0009739F0AC010C
:1034500041505109842395232F5FF7CF822F089580
:103460008091F101843021F11092DB0120E488E1A8
:1034700090E00FB6F894A895809360000FBE20935B
:10348000600080E00E94100883B7817F846083BF62
:1034900083B7816083BF7894889583B78E7F83BF1D
:1034A00088E10FB6F89480936000109260000FBE20
:1034B0000895089508950E94591A0E94A1020E9439
:1034C0005A1A0E94960391E0811101C090E0892F61
:1034D00008950E94B0130E94170F0C94100882E008
:1034E00084BD93E095BD9AEF97BD80936E000895DB
:1034F0002FB7F8948091DC019091DD01A091DE015D
:10350000B091DF012FBF0895CF92DF92EF92FF922B
:103510000F931F932FB7F8944091DC015091DD0178
:103520006091DE017091DF012FBF6A017B01EE2403
:10353000FF248C0120E030E0C016D106E206F3063D
:1035400010F4415051099A01281B390BC9011F91F0
:103550000F91FF90EF90DF90CF9008951F920F9200
:103560000FB60F9211248F939F93AF93BF938091C7
:10357000DC019091DD01A091DE01B091DF010196A7
:10358000A11DB11D8093DC019093DD01A093DE01AC
:10359000B093DF01BF91AF919F918F910F900FBEBC
:1035A0000F901F9018950E94140CF8942FEF87EA43
:1035B00091E6215080409040E1F700C0000087E094
:1035C00090EBDC018093FB019093FC01A093FD0143
:1035D000B093FE019CE088E10FB6F894A895809323
:1035E00060000FBE90936000FFCFEF92FF920F93A9
:1035F0001F93CF93DF93D82FCDE08C2F0E948F03A2
:1036000005E010E0E82EF12CC701002E02C09595D0
:1036100087950A94E2F780FF09C0602F7C2F80E035
:103620000E942005D81302C081E006C00150110994
:1036300058F7C15010F780E0DF91CF911F910F91A3
:10364000FF90EF900895CF93C82F8CE20E94F51A57
:10365000882321F08C2FCF910C94F51A80E0CF9124
:103660000895CF930E94781C811102C00E945E1CB5
:10367000C5E6C15049F00E94A1028FE39CE9019781
:10368000F1F700C00000F5CF89E20E94231B8111F1
:1036900013C18AE20E94231B81110E945E1C85E0F7
:1036A0000E94231B81110E94D31A0E94831C8093C5
:1036B000DA0187E00E94231B8823A9F18BE10E9495
:1036C000231B882351F08091DA0181FB222720F906
:1036D00091E0922790FB81F90EC08EE00E94231B9F
:1036E000882361F08091DA0182FB222720F991E0A2
:1036F000922790FB82F98093DA0115C080E10E9445
:10370000231B9091DA01882341F093FB222720F9B3
:1037100081E0822780FB93F904C0892F809580FB8C
:1037200090F99093DA018091DA010E94871C0E943F
:10373000951C8093FA0180EE0E94231B882341F0A0
:103740008091FA01982F909590FB80F98093FA016F
:1037500089E30E94231B882359F08091FA0181FBA1
:10376000222720F991E0922790FB81F98093FA01BA
:1037700082EE0E94231B882359F08091FA0182FB7C
:10378000222720F991E0922790FB82F98093FA0199
:1037900086EE0E94231B882359F08091FA0183FB57
:1037A000222720F991E0922790FB83F98093FA0178
:1037B00083EE0E94231B882359F08091FA0184FB39
:1037C000222720F991E0922790FB84F98093FA0157
:1037D00085E30E94231B882359F08091FA0185FB21
:1037E000222720F991E0922790FB85F98093FA0136
:1037F00081E30E94231B882359F08091FA0186FB04
:10380000222720F991E0922790FB86F98093FA0114
:1038100081E10E94231B882359F08091FA0187FBE4
:10382000222720F991E0922790FB87F98093FA01F3
:103830008091FA010E94991C8091FA0187FB8827E8
:1038400080F980930D0187E20E94231BC82F8EE12F
:103850000E94231B8111C2608FE10E94231B8111F2
:10386000C46080E20E94231B8111C86081E20E9433
:10387000231B8111C06182E20E94231B8111C0625F
:1038800083E20E94231B8111C06484E20E94231BF7
:10389000882311F0C06802C0CC2329F08C2F0E942D
:1038A000901C6C2F03C00E948C1C682F70E080E07D
:1038B00090E0CF910C947017CF9108956DEE7EEF4C
:1038C00080E090E00E94CA2260E082E090E00E94E6
:1038D000B82260E083E090E00E94B82260E084E0DB
:1038E00090E00E94B82260E085E090E00C94B8225D
:1038F00080E090E00E94B22221E08D3E9E4F09F0D0
:1039000020E0822F089582E090E00C94AA22682F94
:1039100082E090E00C94B82283E090E00C94AA221C
:10392000682F83E090E00C94B82284E090E00C943F
:10393000AA22682F84E090E00C94B8228091E201E2
:1039400080FF0BC06091130185E0689FB0011124D6
:1039500075956795759567952BC081FF09C0609136
:10396000130185E0689FB00111247595679520C00B
:1039700082FF07C06091130185E0689FB0011124A8
:1039800017C09091E3019923D1F06091120196172D
:1039900088F72091130185E0289F90011124929FC0
:1039A000A001939F500D112470E0CA010E947C2257
:1039B0006038710540F46115710539F002C065E0A9
:1039C00070E0862F08958FE7089581E00895809133
:1039D000E20180FF08C06091110170E07595679564
:1039E0007595679521C081FF06C06091110170E057
:1039F0007595679519C082FF04C06091110170E050
:103A000010C09091E3019923C1F0609110019617C5
:103A1000A0F780911101899FC001112470E00E94DC
:103A20007C226038710528F46115710521F0862F1C
:103A300008958FE7089581E0089561E070E0F4CF84
:103A4000803F21F40E949E1C819504C0813F29F48F
:103A50000E949E1C8093E6010895823F21F40E94FB
:103A60009E1C819504C0833F29F40E949E1C809374
:103A7000E5010895893F19F40E94E71C05C08A3FBB
:103A800031F40E94E71C81958093E70108958B3FF4
:103A900021F40E94E71C819504C08C3F29F40E9408
:103AA000E71C8093E8010895843F21F48091E401AC
:103AB000816017C0853F21F48091E401826011C0CC
:103AC000863F21F48091E40184600BC0873F21F49C
:103AD0008091E401886005C0883F31F48091E40161
:103AE00080618093E40108958D3F21F48091E2018B
:103AF00081600BC08E3F21F48091E201826005C09D
:103B00008F3F29F48091E20184608093E20108955F
:103B1000803F39F48091E60187FF6CC01092E60186
:103B200069C0813F29F48091E6011816BCF362C098
:103B30009091E501823F29F497FF5CC01092E50166
:103B400059C0833F19F41916CCF354C0893F41F48E
:103B50008091E70118160CF04DC01092E7014AC0A1
:103B60008A3F29F48091E70187FF44C0F6CF8B3F5D
:103B700039F48091E80187FF3DC01092E8013AC016
:103B80008C3F29F48091E8011816BCF333C0843FC0
:103B900021F48091E4018E7F17C0853F21F480914C
:103BA000E4018D7F11C0863F21F48091E4018B7F79
:103BB0000BC0873F21F48091E401877F05C0883FD7
:103BC00031F48091E4018F7E8093E40113C08D3F36
:103BD00021F48091E2018E7F0BC08E3F21F4809111
:103BE000E2018D7F05C08F3F29F48091E2018B7F38
:103BF0008093E2018091E50181110EC08091E60180
:103C000081110AC08091E701811106C08091E8010D
:103C1000811102C01092E301089584EE91E00E94A8
:103C20002E0F0E94781A9093E1018093E00108958D
:103C30001F93CF93DF938091E0019091E1010E9467
:103C4000841AAC019091E301992321F02091140191
:103C500030E006C0209115018AE0289F90011124D0
:103C60004217530708F486C08091E501C091E60130
:103C7000D091E7011091E801811107C0C11176C010
:103C8000D11174C0111172C075C09F3F19F09F5FB0
:103C90009093E301181624F40E949E1C8093E50182
:103CA0008091E50187FF05C00E949E1C819580934D
:103CB000E5011C1624F40E949E1C8093E60180916D
:103CC000E60187FF05C00E949E1C81958093E60156
:103CD0006091E501662339F1C091E601CC2319F129
:103CE000772767FD7095872F972F0E948D2123E3FB
:103CF00033E343E35FE30E94F1210E945A21609382
:103D0000E5016C2F772767FD7095872F972F0E940D
:103D10008D2123E333E343E35FE30E94F1210E941B
:103D20005A216093E6011D1624F40E94E71C80933B
:103D3000E7018091E70187FF05C00E94E71C81959C
:103D40008093E701111624F40E94E71C8093E80198
:103D50008091E80187FF05C00E94E71C8195809350
:103D6000E801DF91CF911F910C940D1E9F3F09F048
:103D70008ECF96CFDF91CF911F910895E4EEF1E0C1
:103D800085E0DF011D928A95E9F71092E301109218
:103D9000E2010895833081F128F4813059F08230B6
:103DA000D1F00895853009F449C0B8F1863009F49E
:103DB00056C0089580911501262F30E0280F311D3F
:103DC0002F3F310524F4680F6093150108958FEF9C
:103DD00080931501089580911401262F30E0280F5B
:103DE000311D2F3F310524F4680F609314010895AD
:103DF0008FEF80931401089580911301262F30E0F6
:103E0000280F311D2F3F310524F4680F60931301F3
:103E100008958FEF80931301089580911201262F4A
:103E200030E0280F311D2F3F310524F4680F6093D7
:103E3000120108958FEF809312010895809111016E
:103E4000262F30E0280F311D2F3F310524F4680F55
:103E50006093110108958FEF80931101089580916F
:103E60001001262F30E0280F311D2F3F310524F49B
:103E7000680F6093100108958FEF809310010895EB
:103E8000833011F128F4813049F0823091F00895A7
:103E9000853081F120F18630C1F1089580911501BE
:103EA000681720F4861B8093150108951092150160
:103EB000089580911401681720F4861B80931401E3
:103EC000089510921401089580911301681720F449
:103ED000861B809313010895109213010895809119
:103EE0001201681720F4861B809312010895109226
:103EF0001201089580911101681720F4861B8093A8
:103F00001101089510921101089580911001681710
:103F100020F4861B809310010895109210010895DB
:103F20000F931F938D3109F46BC008F03FC08E30A2
:103F300009F47FC0C0F4873009F469C068F48630A2
:103F400009F0B1C08091DA01817F8E7F8093DA0120
:103F500081E08093EA01A8C0883009F4A2C08B30C8
:103F600009F49FC0A0C0863109F49BC078F4803169
:103F700009F472C0813109F096C00E94B01390918B
:103F80000D0181E0892780930D018BC0893109F4EF
:103F900088C08B3109F087C08091DA0181FB22272C
:103FA00020F991E0922790FB81F94CC0853309F408
:103FB00070C048F4873209F46CC008F459C08932E3
:103FC00009F467C070C0833438F48A3308F04EC0F7
:103FD000883309F466C067C0833409F45AC0883452
:103FE00009F061C00E94B0130FEF13ED20E3015000
:103FF00010402040E1F700C000000E94D31A51C0D9
:104000000E9414210E94170F0E9410084AC090912C
:10401000DA01892F8095817080FB90F929F09660F4
:1040200098609093DA0140C0997F977F9093DA016E
:1040300038C08091DA0182FB222720F991E0922793
:1040400090FB82F98093DA01992359F18091DA018A
:1040500081608093DA0125C08091DA0183FB2227F9
:1040600020F991E0922790FB83F9ECCF895301C0AE
:104070008D5141E050E060E070E08A019B0104C096
:10408000000F111F221F331F8A95D2F7C901B801F3
:1040900004C061E070E080E090E00E9470170E9430
:1040A000B01381E001C080E01F910F91089580E07E
:1040B000089580E00895CF93C82F8091EA01813060
:1040C00079F018F08230E9F187C0E0910E01F091AB
:1040D0000F018081813169F0823209F07FC009C00F
:1040E000E0910E01F0910F018081813111F0823257
:1040F00061F48C2F0E945720811104C08C2F0E94E4
:10410000901F1DC081E090E01AC08C2F0E945920A2
:10411000811114C0C43179F048F4CB3079F0C0314A
:1041200009F060C082E08093EA0108C0C93219F04A
:10413000C83321F057C01092EA0154C081E0817069
:1041400053C0C93289F118F5C43171F1A8F4C730F0
:1041500009F046C08AE08093150194E19093140120
:1041600093E0909313018093120188E080931101F2
:1041700088E28093100134C0CE51C63088F5EC2F10
:10418000F0E0E65DFE4F80818093E90129C0CE34E6
:10419000E9F020F4CB3421F56AE013C0C13579F0A1
:1041A000C235F1F461E00DC08091E901882319F076
:1041B0001092E90115C081E08093EA0115C061E029
:1041C00006C08091E9010E94CA1E0AC06AE080917F
:1041D000E9010E94401F04C01092EA0180E004C07F
:1041E00081E002C080E0ABCFCF910895E1E8F0E03C
:1041F0008081886080838081816080838FB7F8941C
:1042000093E09093890090ED909388008FBF08957C
:10421000EFE6F0E08081826080830895EFE6F0E0D1
:1042200080818D7F80830895EFE6F0E0908182E0C9
:104230008927808308951F920F920FB60F92112441
:104240002F933F934F935F936F937F938F939F939E
:10425000AF93BF93EF93FF938091EB019091EC01AB
:1042600001969093EC018093EB01811103C082E0F1
:104270000E941008E091EC01E695E695F0E0E05A26
:10428000FC4FE4918091EB018E1303C080E00E940B
:104290001008FF91EF91BF91AF919F918F917F9106
:1042A0006F915F914F913F912F910F900FBE0F90A3
:1042B0001F90189504D06894B1118DC0089570D0E6
:1042C00088F09F5790F0B92F9927B751A0F0D1F0FF
:1042D000660F771F881F991F1AF0BA95C9F712C089
:1042E000B13081F077D0B1E0089574C0672F782F96
:1042F0008827B85F39F0B93FCCF3869577956795F5
:10430000B395D9F73EF490958095709561957F4F60
:104310008F4F9F4F0895E89409C097FB3EF4909506
:104320008095709561957F4F8F4F9F4F9923A9F08E
:10433000F92F96E9BB279395F6958795779567951D
:10434000B795F111F8CFFAF4BB0F11F460FF1BC061
:104350006F5F7F4F8F4F9F4F16C0882311F096E9F4
:1043600011C0772321F09EE8872F762F05C06623A2
:1043700071F096E8862F70E060E02AF09A95660F5B
:10438000771F881FDAF7880F9695879597F9089514
:1043900057FD9058440F551F59F05F3F71F04795F6
:1043A000880F97FB991F61F09F3F79F087950895DB
:1043B000121613061406551FF2CF4695F1DF08C0FA
:1043C000161617061806991FF1CF86957105610517
:1043D00008940895E894BB2766277727CB0197F9BF
:1043E00008950BD078C069D028F06ED018F09523CE
:1043F00009F05AC05FC01124EECFCADFA0F3959F29
:10440000D1F3950F50E0551F629FF001729FBB27BB
:10441000F00DB11D639FAA27F00DB11DAA1F649F67
:104420006627B00DA11D661F829F2227B00DA11D1A
:10443000621F739FB00DA11D621F839FA00D611DA0
:10444000221F749F3327A00D611D231F849F600DC1
:10445000211D822F762F6A2F11249F5750408AF0FA
:10446000E1F088234AF0EE0FFF1FBB1F661F771F86
:10447000881F91505040A9F79E3F510570F014C01D
:10448000AACF5F3FECF3983EDCF38695779567956E
:10449000B795F795E7959F5FC1F7FE2B880F911DA4
:1044A0009695879597F9089597F99F6780E870E04A
:1044B00060E008959FEF80EC089500240A9416169A
:1044C000170618060906089500240A941216130602
:1044D000140605060895092E0394000C11F4882390
:1044E00052F0BB0F40F4BF2B11F460FF04C06F5FAC
:1044F0007F4F8F4F9F4F089597FB072E16F4009420
:1045000007D077FD09D00E94962207FC05D03EF423
:10451000909581959F4F0895709561957F4F08956F
:10452000EE0FFF1F0590F491E02D0994AA1BBB1B11
:1045300051E107C0AA1FBB1FA617B70710F0A61BA3
:10454000B70B881F991F5A95A9F780959095BC01C4
:10455000CD010895F999FECF92BD81BDF89A9927B2
:1045600080B50895A8E1B0E042E050E00C94D2227A
:10457000262FF999FECF92BD81BDF89A019700B41C
:10458000021639F01FBA20BD0FB6F894FA9AF99ABC
:104590000FBE08950196272F0E94B9220C94B822CD
:1045A000DC01CB01FC01F999FECF06C0F2BDE1BDF3
:1045B000F89A319600B40D9241505040B8F70895E2
:0445C000F894FFCF9D
:1045C40002201208A0087D08490815080101C70146
:1045D40028080A03140A3F4D36392103D4029E02E7
:1045E4006502F80111022A024302010203040506CE
:0445F40007080900AB
:00000001FF
